:100000000C942A000C9447000C943F040C94470075
:100010000C9447000C9447000C9447000C94470044
:100020000C94A2040C9447000C9447000C944700D5
:100030000C9447000C94ED010C9447000C9447007D
:100040000C9447000C9447000C9447000C94470014
:100050000C94470011241FBECFE5D8E0DEBFCDBF12
:1000600010E0A0E6B0E0E2EDF1E102C005900D92F3
:10007000AC3BB107D9F712E0ACEBB0E001C01D9288
:10008000A634B107E1F70E94F2050C94E8080C943D
:100090000000CF93DF93CDB7DEB724970FB6F89467
:1000A000DEBF0FBECDBF69837A838B839C8389813A
:1000B0009A81AB81BC810197A109B10989839A8397
:1000C000AB83BC8389819A81AB81BC810097A105F8
:1000D000B10569F724960FB6F894DEBF0FBECDBF09
:1000E000DF91CF910895CF93DF93CDB7DEB7EBE3E8
:1000F000F0E01082EAE3F0E01082E8E3F0E0108242
:10010000E7E3F0E01082E5E3F0E01082E4E3F0E002
:1001100080EC8083E2E3F0E01082E1E3F0E082E94A
:100120008083EFE4F0E080E18083EEE4F0E081E0C2
:100130008083EDE4F0E01082ECE4F0E01082E7E48C
:10014000F0E01082E6E4F0E01082EBE4F0E01082F0
:10015000EAE4F0E01082E9E4F0E087E08083E8E49C
:10016000F0E08AE28083ABE5B0E0EBE5F0E080818F
:1001700080688C93E5E5F0E088E08083E4E5F0E0DA
:100180001082EAE5F0E080E88083E0E3F0E080813F
:100190009927807290700097B9F0EBE3F0E010823D
:1001A000EAE3F0E01082A2E3B0E0E2E3F0E0908165
:1001B0008CEF89238C93A1E3B0E0E1E3F0E0908140
:1001C0008CEF89238C932EC0A8E3B0E0E8E3F0E045
:1001D00080818B7F8C93A7E3B0E0E7E3F0E0808140
:1001E00084608C93ABE3B0E0EBE3F0E080818F754B
:1001F0008C93AAE3B0E0EAE3F0E08081806A8C931C
:10020000EBE2F0E01082EAE2F0E088E98083E0E4EB
:10021000F0E086E88083E0E4F0E01082E9E2F0E0DC
:1002200083E08083E9E5F0E088E08083E8E2F0E0C5
:1002300080E88083E0E5F0E01082E7E2F0E0108201
:10024000E6E2F0E080E880837894DF91CF91089532
:10025000CF93DF93CDB7DEB721970FB6F894DEBF0B
:100260000FBECDBF8983EBE2F0E0808199278072D9
:1002700090700097C1F3ECE2F0E0898180832196D1
:100280000FB6F894DEBF0FBECDBFDF91CF910895BA
:10029000CF93DF93CDB7DEB722970FB6F894DEBFCA
:1002A0000FBECDBF9A8389830AC0E981FA8180811C
:1002B0000E94280189819A8101969A838983E98124
:1002C000FA818081882389F78DE00E942801229697
:1002D0000FB6F894DEBF0FBECDBFDF91CF9108956A
:1002E000CF93DF93CDB7DEB727970FB6F894DEBF75
:1002F0000FBECDBF6A837B838C839D830BC08A81B5
:100300009B81AC81BD810197A109B1098A839B833F
:10031000AC83BD8380912B0290912C02009741F415
:100320008A819B81AC81BD810097A105B10539F718
:100330008A819B81AC81BD810097A105B10539F40B
:1003400081E090E09093C8008093C7003BC080910B
:100350002F0290913002FC01E75DFE4F808189837E
:1003600080912B0290912C0218161906ACF4809102
:100370002F029091300201969093300280932F02C9
:1003800080912F029091300221E08030920721F479
:100390001092300210922F02F89480912B029091CB
:1003A0002C02181619064CF480912B0290912C0205
:1003B000019790932C0280932B027894898199273E
:1003C0009F838E838E819F8127960FB6F894DEBF20
:1003D0000FBECDBFDF91CF9108951F920F920FB640
:1003E0000F9211242F938F939F93EF93FF93CF93AB
:1003F000DF93CDB7DEB72297DEBFCDBFEBE2F0E0F3
:1004000080818A83ECE2F0E0808189838A81992768
:100410008C7190700097B1F5809122019091230129
:10042000FC01E75DFE4F89818083809122019091DC
:100430002301019690932301809322018091220150
:100440009091230121E08030920721F41092230142
:100450001092220180912B0290912C020196909390
:100460002C0280932B0280912B0290912C0221E090
:100470008030920739F410922C0210922B0281E006
:10048000809327012296F894DEBFCDBFDF91CF91F4
:10049000FF91EF919F918F912F910F900FBE0F9031
:1004A0001F901895CF93DF93CDB7DEB725970FB682
:1004B000F894DEBF0FBECDBF19821A821DC089819C
:1004C0009927FC01EE51FF4F20818A819927FC0179
:1004D000EB59FF4F80811D82281711F081E08D8339
:1004E00089818F5F89839D81992319F01C821B82EA
:1004F0000AC08A818F5F8A838A81853000F381E018
:1005000090E09C838B838B819C8125960FB6F89419
:10051000DEBF0FBECDBFDF91CF910895CF93DF93A4
:10052000CDB7DEB722970FB6F894DEBF0FBECDBFB2
:100530009A8389838091430290914402019690931B
:1005400044028093430222960FB6F894DEBF0FBE9A
:10055000CDBFDF91CF910895CF93DF93CDB7DEB7B5
:1005600024970FB6F894DEBF0FBECDBF1C821B824E
:100570001A82198260EA76E881E090E00E947001B8
:100580008A3031F08091C7009091C800009791F3B4
:1005900060EA76E881E090E00E9470018093420278
:1005A000809142028B3229F489819A8101969A8343
:1005B000898389819A8124960FB6F894DEBF0FBE95
:1005C000CDBFDF91CF9108951F93CF93DF93CDB728
:1005D000DEB729970FB6F894DEBF0FBECDBF1C82E1
:1005E0001B821A8219828FE48D838BE48E83109292
:1005F000C8001092C70060EA76E881E090E00E94AF
:1006000070018D3001F460EA76E881E090E00E94AC
:1006100070018A3001F48091C7009091C800009762
:1006200041F01986188634C089819A8101969A838F
:1006300089832B813C81CE010596FC01E20FF31FDB
:10064000108160EA76E881E090E00E9470011F82EC
:10065000181711F481E08F838B819C8101969C8314
:100660008B839F81992301F760EA76E881E090E02F
:100670000E9470018D3001F460EA76E881E090E03C
:100680000E9470018A3001F489819A819987888754
:100690008885998529960FB6F894DEBF0FBECDBF29
:1006A000DF91CF911F9108951F93CF93DF93CDB723
:1006B000DEB725970FB6F894DEBF0FBECDBF1A8206
:1006C000198260EA76E881E090E00E9470018A3049
:1006D00061F08091C7009091C800009791F305C028
:1006E00089819A8101969A8389838B819C81FC01FF
:1006F000E559FF4F108160E771E181E090E00E94D1
:1007000070011D82181711F481E08D838B819C810B
:1007100001969C838B8381E09D818927882331F416
:100720008091C7009091C8000097D1F260EA76E806
:1007300081E090E00E9470018A3031F08091C70022
:100740009091C800009791F325960FB6F894DEBFFC
:100750000FBECDBFDF91CF911F9108951F93CF930F
:10076000DF93CDB7DEB728970FB6F894DEBF0FBE84
:10077000CDBF1E821D821C821B821A82198260EAF2
:1007800076E881E090E00E9470018A3009F454C05C
:100790008091C7009091C800009789F34DC0809167
:1007A000220190912301009709F45CC060E771E198
:1007B00081E090E00E947001809342028D819E81D1
:1007C000FC01EB58FF4F9081809142029817A1F5F0
:1007D0008D819E8101969E838D838D819E81FC01FA
:1007E000EB58FF4F108160E771E181E090E00E94DB
:1007F00070011817F9F489819A8101969A83898387
:1008000005C08B819C8101969C838B838D819E8109
:1008100001969E838D838D819E81FC01EB58FF4F55
:10082000108160E771E181E090E00E94700118178B
:1008300041F302C01E821D8289819A81009709F4CA
:10084000AECF60E771E181E090E00E9470018A30F4
:10085000C1F71092C8001092C70089819A819887C9
:100860008F8301C002C08F81988528960FB6F894B7
:10087000DEBF0FBECDBFDF91CF911F9108951F92B4
:100880000F920FB60F9211242F933F934F935F93C4
:100890006F937F938F939F93AF93BF93EF93FF9348
:1008A000CF93DF93CDB7DEB71092C2001092C10094
:1008B00010923502109234021CC0E0E3F0E0808117
:1008C000992788709070009739F081E090E09093BC
:1008D000C2008093C10004C01092C2001092C100F7
:1008E0008091340290913502019690933502809365
:1008F0003402809134029091350282339105ECF2FA
:100900008091C1009091C200181619066CF281E026
:1009100090E09093D4008093D3000E94ED04DF9187
:10092000CF91FF91EF91BF91AF919F918F917F9167
:100930006F915F914F913F912F910F900FBE0F904C
:100940001F9018951F920F920FB60F9211242F939C
:100950008F939F93EF93FF93CF93DF93CDB7DEB742
:100960008091C3009091C40001969093C40080933D
:10097000C300ECE4F0E0118210828091D5009091E8
:10098000D600009741F48091C3009091C4002FE0FD
:10099000803A920719F4EFE4F0E01082E0E3F0E02F
:1009A0008081992780729070009739F081E090E003
:1009B0009093D8008093D70004C01092D800109272
:1009C000D700DF91CF91FF91EF919F918F912F9160
:1009D0000F900FBE0F901F901895CF93DF93CDB758
:1009E000DEB7A4E3B0E0E4E3F0E0808180688C93BC
:1009F000A5E3B0E0E5E3F0E0908180E889278C93FF
:100A0000DF91CF910895CF93DF93CDB7DEB7A4E305
:100A1000B0E0E4E3F0E0808180688C93A5E3B0E08F
:100A2000E5E3F0E0808180688C93DF91CF910895B9
:100A3000CF93DF93CDB7DEB7A4E3B0E0E4E3F0E01B
:100A4000808180648C93A5E3B0E0E5E3F0E09081E1
:100A500080E489278C93DF91CF910895CF93DF9322
:100A6000CDB7DEB7A4E3B0E0E4E3F0E080818064DA
:100A70008C93A5E3B0E0E5E3F0E0808180648C93A3
:100A8000DF91CF910895CF93DF93CDB7DEB7A1E388
:100A9000B0E0E1E3F0E0808180688C93A2E3B0E015
:100AA000E2E3F0E0908180E889278C93DF91CF9199
:100AB0000895CF93DF93CDB7DEB724970FB6F894A0
:100AC000DEBF0FBECDBF81E890E00E9448010E94CA
:100AD000E402009719F41A82198213C0E0E4F0E0EE
:100AE0001082E9E2F0E083E080838FE890E00E94EA
:100AF00048010E94E402009719F41A82198201C089
:100B000004C089819A819C838B838B819C812496EC
:100B10000FB6F894DEBF0FBECDBFDF91CF91089521
:100B2000CF93DF93CDB7DEB724970FB6F894DEBF2F
:100B30000FBECDBF84E990E00E9448018FEF9FEF88
:100B40009093BF008093BE008091BE009091BF0043
:100B500001979093BF008093BE008091BE0090915A
:100B6000BF00009789F70E94E402009719F41A82E7
:100B7000198229C01092C8001092C70089E990E03C
:100B80000E9448018FEF9FEF9093BF008093BE00BB
:100B90008091BE009091BF0001979093BF00809319
:100BA000BE008091BE009091BF00009789F70E941F
:100BB000E402009719F41A82198205C01092C80045
:100BC0001092C70004C089819A819C838B838B819A
:100BD0009C8124960FB6F894DEBF0FBECDBFDF9187
:100BE000CF9108951F93CF93DF93CDB7DEB72997A9
:100BF0000FB6F894DEBF0FBECDBF109224011C8249
:100C00001B820E947300EAE3F0E084E0808360E6E8
:100C100073EE86E190E00E944900ABE3B0E0EBE3C5
:100C2000F0E090818BEF89238C93AAE3B0E0EAE3B4
:100C3000F0E090818BEF89238C930E94AE030E9499
:100C400090051092C8001092C700AFE4B0E0EFE446
:100C5000F0E0908180E189278C931A82198205C087
:100C600089819A8101969A83898389819A8125E76E
:100C700080339207ACF3AFE4B0E0EFE4F0E09081B2
:100C800080E189278C93E7E2F0E083E08083A6E2AD
:100C9000B0E0E6E2F0E0808180648C93E6E2F0E090
:100CA00080819927807490700097C1F7E4E2F0E0AA
:100CB000808199279093320280933102E5E2F0E03F
:100CC0008081992790934102809340028091400255
:100CD00090914102982F882790934102809340027F
:100CE0002091400230914102809131029091320274
:100CF000822B932B9093410280934002809140027B
:100D0000909141028233910548F4A1E3B0E0E1E320
:100D1000F0E080818F778C93889507C0A1E3B0E0E5
:100D2000E1E3F0E0808180688C938091D70090911E
:100D3000D800009709F444C0EBE2F0E01082EAE248
:100D4000F0E01082E0E4F0E01082E0E4F0E01082F5
:100D5000E9E2F0E01082EBE3F0E01082EAE3F0E099
:100D60001082A2E3B0E0E2E3F0E090818CEB892313
:100D70008C93A1E3B0E0E1E3F0E090818CEB892378
:100D80008C9380914002909141028333910538F019
:100D9000A1E3B0E0E1E3F0E0808180688C93A8E318
:100DA000B0E0E8E3F0E090818BEF89238C93A7E338
:100DB000B0E0E7E3F0E090818BEF89238C9344C0AF
:100DC000A8E3B0E0E8E3F0E090818BEF89238C9317
:100DD000A7E3B0E0E7E3F0E0808184608C93ABE3CD
:100DE000B0E0EBE3F0E080818F758C93AAE3B0E094
:100DF000EAE3F0E08081806A8C93E2E3F0E0108225
:100E0000E1E3F0E082E18083809140029091410231
:100E10008333910538F0A1E3B0E0E1E3F0E08081B5
:100E200080688C93EBE2F0E01082EAE2F0E088E97F
:100E30008083E0E4F0E086E88083E0E4F0E0108284
:100E4000E9E2F0E083E08083E0E3F0E0808199274D
:100E500080749070009749F48091CD009091CE00FD
:100E600001969093CE008093CD0080912B029091BB
:100E70002C02009709F48CC010922401E0E3F0E00A
:100E800080819927807490700097D1F48091D90067
:100E90009091DA00009739F481E090E09093DC00C3
:100EA0008093DB000DC08091CD009091CE00019623
:100EB0009093CE008093CD001092D6001092D50072
:100EC0000E94AC02009709F048C0109224010FC0A4
:100ED00080912401282F332783EA90E0F901EE5115
:100EE000FF4F8083809124018F5F80932401809144
:100EF0002401803468F310922401809142028A30E8
:100F000071F030912401832F992720914202FC0136
:100F1000EE51FF4F2083832F8F5F8093240160EA7F
:100F200076E881E090E00E94700180934202809117
:100F300042028A3071F030912401832F9927209149
:100F40004202FC01EE51FF4F2083832F8F5F80937D
:100F50002401809142028A3011F70E9452028823B4
:100F6000B9F08091CD009091CE00009789F08091EA
:100F7000CB009091CC0001969093CC008093CB0055
:100F8000AFE4B0E0EFE4F0E0908180E189278C935A
:100F90008091D3009091D400009709F4A8C080916B
:100FA000CB009091CC00009709F4A1C01092D4001E
:100FB0001092D3001092CC001092CB0010928000BF
:100FC00010927F00EFE4F0E0108284EA90E00E944B
:100FD00048018FEF9FEF9093BF008093BE008091F8
:100FE000BE009091BF0001979093BF008093BE0018
:100FF0008091BE009091BF00009789F78091CF004B
:101000009091D00001969093D0008093CF0008C0BB
:101010008091C5009091C6009093C6008093C50052
:1010200060EA76E881E090E00E9470018A3081F702
:1010300009C08091C9009091CA0001969093CA009E
:101040008093C9008091C5009091C60099878887D8
:10105000E885F985ED59FF4F108160EA76E881E077
:1010600090E00E9470011F82181711F491E09F8395
:101070008885998501969093C6008093C5002F813D
:101080002223B9F608C08091C5009091C6009093C4
:10109000C6008093C50060EA76E881E090E00E9497
:1010A00070018A3081F788EA90E00E9448018FEF52
:1010B0009FEF9093BF008093BE008091BE009091FF
:1010C000BF0001979093BF008093BE008091BE0047
:1010D0009091BF00009789F70E94E402009719F4ED
:1010E0001E821D8269C01092C8001092C7008091B4
:1010F000D3009091D4000097B9F18091CF009091E6
:10110000D000009789F182EB90E00E9448018FEFB8
:101110009FEF9093BF008093BE008091BE0090919E
:10112000BF0001979093BF008093BE008091BE00E6
:101130009091BF00009789F70E94E402009719F48C
:101140001E821D8239C01092C8001092C7001092F2
:10115000D0001092CF008091D1009091D2000196E2
:101160009093D2008093D1008091D3009091D400CD
:101170000097F1F08091D1009091D2000097C1F0DA
:101180000E9454031092D4001092D3001092D20007
:101190001092D100A4E3B0E0E4E3F0E08081806C41
:1011A0008C93A5E3B0E0E5E3F0E080818F738C934E
:1011B00084E68093240167CD8D819E8129960FB6A8
:1011C000F894DEBF0FBECDBFDF91CF911F91089580
:0211D000FFCF4F
:1011D2000300F04F4B52494E470D004E4F20434102
:1011E20052524945524361206C2052656164790133
:1011F2000041542B4950523D31313532303000419B
:1012020054265700415445300041542B434D474624
:101212003D3100004154410041542B434846413D79
:0C122200300041542B434846413D310050
:00000001FF
